:100000000C9466000C9485000C9485000C9485007B
:100010000C9485000C9485000C94C6010C9485000A
:100020000C9485000C9485000C9485000C9485003C
:100030000C9485000C9485000C9485000C9485002C
:100040000C94DF080C9485000C9485000C948500BA
:100050000C9485000C9485000C9485000C949E08EB
:100060000C9485000C9485000C941B060C94850060
:100070000C9485000C9485000C9485000C948500EC
:100080000C9485000C9485000C9485000C948500DC
:100090000C94F4090C94D7050C9485000C948500FD
:1000A0000C9485000C9485000C9481010C948500BF
:1000B0000C9485000C9485000C9485000C948500AC
:1000C0000C9485000C9485000C94850011241FBEAF
:1000D000CFEFD1E2DEBFCDBF18E0A0E0B2E0EEE4AA
:1000E000F0E200E00BBF02C007900D92AC36B10702
:1000F000D9F71DE0ACE6B8E001C01D92A736B10704
:10010000E1F70E946B0D0C9425100C94000089EB14
:1001100096E2A0E0B0E08093FD099093FE09A093E1
:10012000FF09B093000A1092010A52E05093020AAC
:1001300031E03093030A83E08093040A1092050AA9
:100140001092060A3093070A1092080A1092090AC0
:100150004FEF40930A0A20E120930B0A30930C0AD8
:1001600088E998E090930E0A80930D0A10920F0A86
:100170004093100A2093110A3093120A9093140AA4
:100180008093130A2093150A5093160A3093170A86
:100190001092180A08958A3010F48093010A089585
:1001A0008A3010F48093020A0895AF92BF92CF92E2
:1001B000DF92FF920F931F93CF93DF936C0180E048
:1001C00090E0F601E80FF91F108201968131910548
:1001D000C1F700E010E098ECA92EB12C23C00E94DA
:1001E000620381E06F2D0E947903C5010197F1F749
:1001F00086E00E94F303282F2F713881832F90E02F
:10020000820F911D8F3F910514F4230F2883F394DF
:1002100021968BE1F81619F7A8950F5F1F4F04364A
:10022000110521F0E6018BE0F82ED9CF80E1DF91B6
:10023000CF911F910F91FF90DF90CF90BF90AF9023
:10024000089581E080937308809171088F5F809397
:1002500071080E946203E091010A80915809F0E060
:1002600024E0EE0FFF1F2A95E1F7E80FF11DEC5394
:10027000FD4F82E060810E94790388EE93E0019750
:10028000F1F786E00E94F303682F6F71609378089E
:100290008AE798E00E945209682F8093790880913C
:1002A0007A0890917B08A0917C08B0917D0880939A
:1002B000740890937508A0937608B093770880919E
:1002C000030A90917808813051F48091040A8917CB
:1002D00078F4809172088F5F809372080EC08091CD
:1002E000040A891728F4809172088F5F809372083E
:1002F0008AE798E070E00E947003A8951092730856
:1003000008951F920F920FB60F920BB60F92112401
:100310002F933F934F935F936F937F938F939F930D
:10032000AF93BF93EF93FF931092A5001092A40098
:100330000E9421012091220230912302E091020AC1
:1003400080915809F0E044E0EE0FFF1F4A95E1F775
:10035000E80FF11DEC5DFD4F8081280F311D3093BA
:10036000A9002093A800FF91EF91BF91AF919F91B9
:100370008F917F916F915F914F913F912F910F904E
:100380000BBE0F900FBE0F901F9018951F920F92EB
:100390000FB60F920BB60F9211242F933F934F93EA
:1003A0005F936F937F938F939F93AF93BF93EF93DD
:1003B000FF93A8958FE00E94F303982F8091730814
:1003C000882309F085C092FF07C086E00E94F303EE
:1003D0008F71809352097CC093FF7AC08091560937
:1003E00090915709029799F4E091010A8091580978
:1003F000F0E074E0EE0FFF1F7A95E1F7E80FF11DD2
:10040000EC53FD4F81E060810E94790361C086EE6C
:1004100098E062E643E559E025E539E00E9474047E
:1004200080935409882309F453C080915509813081
:1004300009F04EC0209174083091750840917608FB
:10044000509177088091E6089091E708A091E8081C
:10045000B091E90882179307A407B507C9F5809101
:10046000EA088830A8F5809158098F3088F4E09127
:10047000010A80915809F0E064E0EE0FFF1F6A95D1
:10048000E1F7EC53FD4FE80FF11D82E061810CC0F4
:10049000E091010AF0E054E0EE0FFF1F5A95E1F7FA
:1004A000EC53FD4F82E060810E9479038091EA085D
:1004B000873019F410926E080BC086EE98E06091B8
:1004C00052094091530920E00E94A20980935409E7
:1004D000FF91EF91BF91AF919F918F917F916F911C
:1004E0005F914F913F912F910F900BBE0F900FBED8
:1004F0000F901F901895DF93CF9300D000D0CDB709
:10050000DEB788E492E0A0E0B0E089839A83AB8311
:10051000BC83CE01019660E070E044E050E00E94B0
:100520000D108DEF99E064E070E04CE150E00E9426
:100530000D100F900F900F900F90CF91DF910895B5
:10054000EF92FF920F93DF93CF93CDB7DEB768970B
:100550000FB6F894DEBF0FBECDBF19821A821B8280
:100560001C820E948700CE01019660E070E044E0AA
:1005700050E00E94FD0F89819A81AB81BC81E5E04A
:10058000EE2EF12CEC0EFD1E88549240A040B0409F
:10059000D1F48DEF99E064E070E04CE150E00E940E
:1005A000FD0F80E092E00E94D2072091FD0930917A
:1005B000FE094091FF095091000AC701B90140E0CE
:1005C00020E001E018C080E192E00E94D20769813A
:1005D0007A81C70140E020E001E00E945F06C70188
:1005E0000E94D20780E292E00E94D207C70168E42D
:1005F00072E040E020E00E945F06C7010E94D2073F
:100600008DE092E00E94D20768960FB6F894DEBFA4
:100610000FBECDBFCF91DF910F91FF90EF90089566
:100620008CE390E090932302809322020E94A00228
:100630008091010A8A3010F48093010A0E949E037F
:10064000E091010A80915809F0E0A4E0EE0FFF1F4D
:10065000AA95E1F7E80FF11DEC53FD4F82E06081B0
:100660000E94790385E06FE040E020E00E941704DB
:100670000E943D030E94990808951092A5001092CF
:10068000A4001092A00085E08093A1008FEF90E07D
:100690009093A9008093A800E2E7F0E08081826057
:1006A00080837894089594B7977F94BFE0E6F0E054
:1006B00090819861908387708860808384B7877FFA
:1006C00084BF0895809158098F3030F48091580983
:1006D0008F5F8093580902C01092580980E00895F6
:1006E0009C01862FB9010E94CC042C9A2C9880E0A2
:1006F00008951F93182F262F88E06FE140E00E9495
:100700001704812F90E09093570980935609113078
:1007100019F482E066E008C085E060E847E021E087
:100720000E94170482E069E00E94E4038EE06CE01E
:100730000E94E403789480E01F9108950F931F9323
:1007400084E00E94BF030CEF13E0C8010197F1F7AA
:1007500017982C988CE090E00197F1F7179A82E0B7
:1007600068E00E94E403C8010197F1F781E06FE1BE
:1007700040E00E94040480E01F910F9108950F9AB9
:10078000249A95B1936095B994B1976094B92398E0
:1007900090E59CBD9CB59C7F9CBD9DB59E7F9DBDFD
:1007A0002CB5982F9370922B9CBD9DB58695869500
:1007B0008170982B9DBDEAE6F0E080818C6080839B
:1007C00080E28CBBED9A0895806C9FB7F8942898CE
:1007D0008EBD0DB407FEFDCF6EBD0DB407FEFDCF7F
:1007E000289A9FBF08958F7380689FB7F8942898C0
:1007F0008EBD0DB407FEFDCF8EBD0DB407FEFDCF3F
:100800008EB5289A9FBF0895FF920F931F93062FCE
:10081000F42E0E94F303082310E002C015950795FB
:10082000FA94E2F7802F1F910F91FF900895DF92C5
:10083000EF92FF920F931F93D82EF62EE42E022FE5
:100840000E94F3036F2D6095682310E002C0000F33
:10085000111FEA94E2F7F0226F298D2D0E94E40324
:100860001F910F91FF90EF90DF900895CB010895B5
:10087000FC01DA015FB7F894289880E28EBD0DB4D0
:1008800007FEFDCF1EBC0DB407FEFDCF4EB56417AD
:1008900030F1942F20E030E01EBC0DB407FEFDCFF8
:1008A0008EB52827022E2295207F2025032E322F59
:1008B00022952F700226269532272327220F220FFA
:1008C000220F20258083915011F03196E5CF1097AB
:1008D00039F01C92232B21F481E08C9301C04068F5
:1008E000289A5FBF842F0895FF920F931F93CF9391
:1008F000DF938C01EA01D901FFB6F894289880E2D1
:100900008EBD0DB407FEFDCF1EBC0DB407FEFDCF9E
:100910009EB5691708F436C020E030E040E050E0B2
:10092000692F70E01CC01EBC0DB407FEFDCF8EB554
:10093000F801E20FF31F80834827042E4295407F81
:100940004025052E542F42954F7004264695542776
:100950004527440F440F440F40252F5F3F4F261774
:10096000370708F3109729F01C92452B11F481E00A
:100970008C93209741F01EBC0DB407FEFDCF8EB5C1
:10098000888301C09068289AFFBE892FDF91CF919C
:100990001F910F91FF900895982FFB012FB7F894A6
:1009A000289880E68EBD0DB407FEFDCF9EBD0DB428
:1009B00007FEFDCF80818EBD915011F03196F7CFAB
:1009C0000DB407FEFDCF289A2FBF0895FC01DA0170
:1009D0003FB7F894289880E28EBD0DB407FEFDCF96
:1009E0001EBC0DB407FEFDCF2EB56217A0F0922FEE
:1009F0001EBC0DB407FEFDCF8EB58083915011F063
:100A00003196F6CF109741F01EBC0DB407FEFDCF16
:100A10008EB58C9301C02068289A3FBF822F08951D
:100A2000833309F080E0089583E30895E82FF0E030
:100A3000EE0FFF1FE15EF54F20813181C90108955E
:100A4000E82FF0E0EE0FFF1FE15EF54F11821082FC
:100A500008959B01AC01529A53985A9A5B9A64E0AC
:100A6000220F331F441F551F6A95D1F760E072E1D2
:100A70008AE790E00E94910F215030401092CD0003
:100A80002093CC0080E48093C80088E98093C9005B
:100A900086E08093CA00789408959B01AC01689A1F
:100AA0006998709A719A74E0220F331F441F551F82
:100AB0007A95D1F760E072E18AE790E00E94910FA9
:100AC000215030401092C5002093C40080E48093F0
:100AD000C00088E98093C10086E08093C2007894CA
:100AE0000895FC0180911C0A8823D1F4F0931E0A1A
:100AF000E0931D0A60931C0A2091210A3091220A7A
:100B0000808190E0822793279093220A8093210A84
:100B100080818093CE008091C90080628093C9005B
:100B200080911C0A8823E1F70895FC018091190A3D
:100B30008823D1F4F0931B0AE0931A0A6093190AF0
:100B400020911F0A3091200A808190E0822793270C
:100B50009093200A80931F0A80818093C600809121
:100B6000C10080628093C1008091190A8823E1F757
:100B70000895DF93CF930F92CDB7DEB78983CE016F
:100B8000019661E00E9495050F90CF91DF91089545
:100B9000DF93CF930F92CDB7DEB78983CE01019655
:100BA00061E00E9471050F90CF91DF9108951F922F
:100BB0000F920FB60F920BB60F9211242F933F9303
:100BC0008F939F93EF93FF93E0911D0AF0911E0A7C
:100BD0003196F0931E0AE0931D0A319780911C0A0A
:100BE000815080931C0A80911C0A882391F0809187
:100BF000210A9091220A2181332727FD3095282749
:100C000039273093220A2093210A81818093CE00D4
:100C100005C08091C9008F7D8093C900FF91EF913D
:100C20009F918F913F912F910F900BBE0F900FBE10
:100C30000F901F9018951F920F920FB60F920BB640
:100C40000F9211242F933F938F939F93EF93FF93D2
:100C5000E0911A0AF0911B0A3196F0931B0AE09377
:100C60001A0A31978091190A81508093190A80914C
:100C7000190A882391F080911F0A9091200A2181FE
:100C8000332727FD3095282739273093200A2093D2
:100C90001F0A81818093C60005C08091C1008F7DAD
:100CA0008093C100FF91EF919F918F913F912F9180
:100CB0000F900BBE0F900FBE0F901F901895BF9214
:100CC000CF92DF92EF92FF920F931F93DF93CF9318
:100CD000CDB7DEB72C970FB6F894DEBF0FBECDBFF1
:100CE0006C01FB01B42EE22E77FD02C0FF2408C088
:100CF000F095E195FF4F8DE2D6018C93FF24F3949C
:100D000040E08E010F5F1F4F10C0200F311FCF0139
:100D10006AE070E00E947E0F805DD9018C93CF0164
:100D20006AE070E00E947E0FFB01242F30E04F5FED
:100D3000EA30F10554F7020F131F8E2F805DF80182
:100D40008083642FCE01019620E305C0FC01E60FED
:100D5000F11D20836F5FE616C8F76B15B8F3862F79
:100D600090E09E012F5F3F4FF901E80FF91F1082BD
:100D70000197D901A80FB91F019640E050E08C01FE
:100D80002E2D30E07EE214C0C801841B950B821723
:100D9000930729F4F601EF0DF11D7083F394F6012A
:100DA000EF0DF11D8C918083F3944F5F5F4F11978E
:100DB000461750F3F601EF0DF11D1082C6012C9677
:100DC0000FB6F894DEBF0FBECDBFCF91DF911F915C
:100DD0000F91FF90EF90DF90CF90BF9008954F92CA
:100DE0005F926F927F928F929F92AF92BF92CF92BB
:100DF000DF92EF92FF920F931F93DF93CF93CDB7C4
:100E0000DEB72C970FB6F894DEBF0FBECDBF3C0106
:100E10006A017B01422E502E77FD02C099240DC03D
:100E2000F094E094D094C094C11CD11CE11CF11C3E
:100E30008DE2F30180839924939488245E010894C1
:100E4000A11CB11C19C00A0D1B1DC701B6012AE067
:100E500030E040E050E00E94B30F605DF801608335
:100E6000C701B6012AE030E040E050E00E94B30F35
:100E7000C901DA016C017D01082D10E08394FAE0CC
:100E8000CF16D104E104F104F4F6A00EB11E8C2DAE
:100E9000805DF5018083482DCE01019620E305C0D9
:100EA000FC01E40FF11D20834F5F5416C8F7441571
:100EB000B8F3842F90E09E012F5F3F4FF901E80FB8
:100EC000F91F10820197D901A80FB91F019620E0E0
:100ED00030E0BC01052D10E05EE214C0CB01821BA6
:100EE000930B8017910729F4F301E90DF11D50834D
:100EF0009394F301E90DF11D8C91808393942F5FFE
:100F00003F4F1197241750F3F301E90DF11D1082A3
:100F1000C3012C960FB6F894DEBF0FBECDBFCF91A4
:100F2000DF911F910F91FF90EF90DF90CF90BF90D6
:100F3000AF909F908F907F906F905F904F900895AB
:100F4000DC010D900020E9F71197A81BB90B6A2F5F
:100F50000E9495050895EF92FF920F93DF93CF9330
:100F6000CDB7DEB72A970FB6F894DEBF0FBECDBF60
:100F7000BC017E010894E11CF11CC70140E020E0A7
:100F800001E00E945F06C7010E94A0072A960FB6E3
:100F9000F894DEBF0FBECDBFCF91DF910F91FF90D0
:100FA000EF900895DC010D900020E9F71197A81B40
:100FB000B90B6A2F0E9471050895CF92DF92EF92CC
:100FC0000F93DF93CF93CDB7DEB72A970FB6F89480
:100FD000DEBF0FBECDBFAB01BC016E010894C11CCA
:100FE000D11CC60120E000E0EE24E3940E94EF064D
:100FF000C6010E94D2072A960FB6F894DEBF0FBE34
:10100000CDBFCF91DF910F91EF90DF90CF900895FA
:10101000EF92FF920F93DF93CF93CDB7DEB72A976E
:101020000FB6F894DEBF0FBECDBFBC017E010894A1
:10103000E11CF11CC70140E020E001E00E945F06D6
:10104000C7010E94D2072A960FB6F894DEBF0FBEE2
:10105000CDBFCF91DF910F91FF90EF900895109247
:10106000800082EC8093810010928200EFE6F0E035
:1010700080818062808378940895FC018081860F4E
:1010800080830895FC018081819580830895FC010F
:101090008081860F80830895FC0180818195808303
:1010A0000895FC0180819181860F971F9183808331
:1010B0000895FC0180819181909581959F4F918346
:1010C00080830895FC0180819181860F971F918311
:1010D00080830895FC0180819181909581959F4F37
:1010E000918380830895FC01882777FD8095982F50
:1010F0002081318142815381260F371F481F591F9C
:1011000020833183428353830895FC018081918140
:10111000A281B381B095A095909581959F4FAF4FD7
:10112000BF4F80839183A283B3830895279A2F981A
:1011300008952F9A08952F98089508951F920F9259
:101140000FB60F9211242F933F938F939F9380910B
:10115000FA09882339F48091FB099091FC0996954E
:10116000879502C08091FA0986BD8091FB09909114
:10117000FC0920916A0830916B0801969093FC0954
:101180008093FB0901978217930729F41092FC09B9
:101190001092FB0915BC9F918F913F912F910F9059
:1011A0000FBE0F901F9018958093FA0970936B08EB
:1011B00060936A0882E085BD80E888BD08951F922B
:1011C0000F920FB60F920BB60F9211242F933F93ED
:1011D0004F936F937F938F939F93AF93BF93EF93AF
:1011E000FF936091860070918700809168099091CB
:1011F00069099B01281B390B40916A098BE0293B47
:10120000380730F14093640910926A098091FD0912
:101210009091FE09A091FF09B091000A80937F0B85
:101220009093800BA093810BB093820B81E080930D
:10123000830B8091970B9091980B01969093980B4C
:101240008093970B82E08093DE078091080A14C098
:10125000483090F4E42FF0E0C901880F991F820F05
:10126000931F84599141EE0FFF1FE957F44F91836B
:1012700080834F5F40936A0970936909609368099E
:10128000FF91EF91BF91AF919F918F917F916F915E
:101290004F913F912F910F900BBE0F900FBE0F906B
:1012A0001F9018959C012F9880916509909166096F
:1012B0000196909366098093650980916709813052
:1012C000E9F48091DF078130C9F480915F098823B8
:1012D000A9F08FEF8093850B80915F098093860B37
:1012E00010925F098091860B8533A1F41092860BD2
:1012F0001092DF0783E780935F090CC08091DF07BE
:10130000813041F48091850B8F3F21F41092860B40
:1013100010925F09D901EFE7FBE08CE101900D929B
:101320008150E1F78091F709860F8093F70980914A
:10133000F809882329F08091F80981508093F809F1
:101340008CE10895FC012F9A6093F8094093F90904
:1013500084818330E9F4ABE5BDE08CE001900D922F
:101360008150E1F781E0809361098091600D8032C6
:1013700068F4E091600DF0E08091610D9091620D54
:10138000EE0FFF1FE55EF24F9183808381E01EC068
:101390008430F1F4ABE5BBE084E201900D92815022
:1013A000E1F78091600B8C3070F48091600B90E0DD
:1013B000B5E0880F991FBA95E1F78556944F63E61B
:1013C0007BE00E94F60F81E08093610980936209BF
:1013D0008CE0089584E693E00E94D2070895F89483
:1013E00080E00E945303FFCF1F920F920FB60F921F
:1013F0000BB60F9211241F932F933F934F935F933C
:101400006F937F938F939F93AF93BF93EF93FF93CC
:101410001091CE00809170098093710980916F09BD
:101420008093700990916E0990936F0920916D09D6
:1014300020936E0910936D09823B41F4953A31F483
:10144000253621F41B3411F40E94EF094091F6096E
:10145000442309F04AC0143471F48091F4098434AF
:10146000D1F51093F50910926C0910926B0981E087
:101470008093F6098EC0133531F48091F4098335D9
:1014800051F581E007C0133741F48091F4098337A7
:1014900011F582E0809360097CC0123539F48091A7
:1014A000F4098235C1F40E94EF0973C0153639F48E
:1014B0008091F409853679F40E947B026AC01D365A
:1014C00051F48091F4098D3631F410925F0981E076
:1014D000809367095EC080915F09882309F059C035
:1014E00010935F091092F60954C08091F509843475
:1014F00009F04BC01092670920916B0930916C097B
:10150000A12FB0E0E42FF0E04C31C0F4A227B327C4
:10151000B070AA0FBB1FAF5EBB4F232F33278D9137
:101520009C918227932790936C0980936B09EF58C5
:10153000F64F10834F5F4093F6092BC0A227B327C5
:10154000B070AA0FBB1FAF5EBB4F832F99272D91A1
:101550003C918227932790936C0980936B09DF015C
:10156000119742E759E0FD01E40FF51F1083892B25
:1015700061F42FE73BE0C901BA01AD010E94E20F1F
:1015800081E08093DE078091090A1092F60910929B
:10159000F5091093F409FF91EF91BF91AF919F91DD
:1015A0008F917F916F915F914F913F912F911F91FB
:1015B0000F900BBE0F900FBE0F901F9018950F93BA
:1015C000FC0101900020E9F73197E81BF90BDB01E2
:1015D0006D917C918E0F9F1F40E020E001E00E9402
:1015E0005F060F9108950F93FC0101900020E9F729
:1015F0003197E81BF90BDB016D917C918E0F9F1FDA
:1016000040E020E001E00E945F060F9108950F93F3
:10161000FC0101900020E9F73197E81BF90BDB0191
:101620006D917C918E0F9F1F40E020E001E00E94B1
:101630005F060F9108950F93DC010D900020E9F7EC
:101640001197A81BB90BFB016081772767FD709587
:101650008A0F9B1F40E020E001E00E945F060F918F
:1016600008950F93FC0101900020E9F73197E81BE2
:10167000F90BDB016C918E0F9F1F70E040E020E0C2
:1016800001E00E945F060F9108958F929F92AF92A2
:10169000BF92CF92DF92EF92FF920F931F93DF934F
:1016A000CF93CDB7DEB7A0970FB6F894DEBF0FBECD
:1016B000CDBF282F198240915A0990915909A92F1D
:1016C000B0E0FD01EC52F84FE081BE2EB40E8091E7
:1016D000160A882319F481E08093160A233309F44B
:1016E0006AC0243338F4213309F4ACC0223309F042
:1016F000BCC013C0263329F1283321F0243309F06C
:10170000B4C060C0442311F0415012C0A752B84F7A
:101710008C91815080935A0910C0242F30E0A75239
:10172000B84F8C9190E001972817390724F44F5F48
:1017300040935A0902C010925A09B0905A09BE0E3D
:1017400094C0AB2DB0E0FD01EF5EF94FE081E230D7
:10175000F9F0E33030F4EE23D9F0E13009F085C040
:1017600008C0E430F9F0E430E8F0E53009F07DC07D
:1017700022C0AA0FBB1FA85DB94FED91FC918081DB
:101780009181A281B3818C509E4FAF4FBF4F4BC010
:10179000AA0FBB1FA85DB94FED91FC91808191818B
:1017A0000A9630C0AA0FBB1FA85DB94FED91FC91FE
:1017B00080818F5F45C0943010F49F5F46C01092C7
:1017C000590949C0AB2DB0E0FD01EF5EF94FE08152
:1017D000E23079F0E33030F4EE2359F0E13009F0F3
:1017E00044C013C0E43021F1E43010F1E530E9F5F4
:1017F00029C0AA0FBB1FA85DB94FED91FC91808154
:1018000091810A979183808330C0AA0FBB1FA85D86
:10181000B94FED91FC9180819181A281B381845F68
:101820009140A040B04080839183A283B3831DC0C8
:10183000AA0FBB1FA85DB94FED91FC91808181502B
:10184000808313C0992321F091509093590903C0CC
:1018500084E08093590910925A09E0915909F0E007
:10186000EC52F84FB080B0925B090B2D10E0209144
:101870005B098091160A90E0820F911D019708176D
:1018800019074CF08091160A2B2D281B822F8F5F91
:1018900080935B0904C0B21610F4B0925B0988E92A
:1018A00093E00E94D207E0915909F0E0EC52F84F22
:1018B000208181E090E0821B9109800F911F0E949E
:1018C00008088CE993E00E94D207E0915909F0E002
:1018D000E752F84F808190E00E9408088EE993E07B
:1018E0000E94D207E0915909F0E0EE0FFF1FE65386
:1018F000F84F808191810E94D20780EA93E00E9494
:10190000D20785EA93E00E94D207E0915909F0E0FE
:10191000EE0FFF1FE653F84F6081718187E29BE075
:101920000E94F60F00E010E0C8018D5D954F6DEB51
:1019300073E00E94F60F065E1F4F31E0043013077C
:1019400099F7A0905B097E010894E11CF11CFAE173
:101950008F2E912C89C01982BA1429F4C7016FEB1C
:1019600073E00E94EB0F8601000F111FF801EB5886
:10197000F84F60817181C7010E94EB0FC70161ECD4
:1019800073E00E94EB0FF601EF5EF94FE081E23069
:1019900001F1E33028F4EE2351F0E130C1F510C03D
:1019A000E43039F1E430F0F0E53089F52BC0085D22
:1019B000194FF80160817181C7010E94F30A27C0A5
:1019C000085D194FF80160817181C7010E94DF0A2B
:1019D0001EC0085D194FF80160817181C7010E9426
:1019E000070B15C0085D194FF80160817181C701AF
:1019F0000CC0085D194FF80160817181C7010E9418
:101A00001B0B05C0C70169E579E00E94310B83EC2F
:101A100093E00E94D20780915B099601281B31094F
:101A2000C9010E9408088EE993E00E94D207C7010D
:101A30000E94D20787EC93E00E94D20780915B0955
:101A4000F601E81BF109EA30F1056CF4188EE89D07
:101A5000C001E99D900DF89D900D11248D5D954F6D
:101A6000B7010E94F60FA394CA2CDD242091160A18
:101A700080915B0990E0820F911DC816D906A4F4ED
:101A800036E13A1588F0E0915909F0E0DF01A752FC
:101A9000B84F2C91EC52F84F808190E0820F911D4D
:101AA000C816D9060CF457CF85EA93E00E94D207F6
:101AB000A0960FB6F894DEBF0FBECDBFCF91DF91D9
:101AC0001F910F91FF90EF90DF90CF90BF90AF905C
:101AD0009F908F9008954F925F926F927F928F9216
:101AE0009F92AF92BF92CF92DF92EF92FF920F93AD
:101AF0001F93DF93CF93CDB7DEB760970FB6F894FF
:101B0000DEBF0FBECDBF279A2F982F9A8FEF8093FD
:101B1000FA098FEF90E090936B0880936A0882E057
:101B200085BD80E888BD80E090E0FC01EE0FFF1FDE
:101B3000E957F44F11821082019680319105A9F77F
:101B400080E090E0FC01EE0FFF1FE55EF24F118296
:101B50001082019680329105A9F780E090E020E89C
:101B60000FB6F89420936100809361000FBE399AFC
:101B7000419A54985C9A60E076E980E090E00E9497
:101B800029058AEC93E00E94D20784E693E00E9444
:101B9000D2071092630B80E090E02EE2FC01A5E0FA
:101BA000EE0FFF1FAA95E1F7E556F44F208311824F
:101BB00001968C30910591F70E942F080E94100326
:101BC0008091FD099091FE09A091FF09B091000A52
:101BD00080937F0B9093800BA093810BB093820B2B
:101BE00081E08093830BF8EC6F2E712C44244A948F
:101BF000EFEF8E2E912C72E0572E6E010894C11CCF
:101C0000D11C61E1A62EB12CAC0EBD1E1092F909BB
:101C10001092F80980ED97E0F3013197F1F7019701
:101C2000D9F780916209882331F18091060A8F3FAC
:101C300079F09091F9098091060A891748F010927D
:101C4000FA0988EE93E090936B0880936A0810C0BD
:101C50008091050A8F3F79F09091F8098091050AEB
:101C6000891748F04092FA0990926B0880926A08AE
:101C700055BC80E888BD8091DF07882321F510914D
:101C80005F0910925F09153321F481E08093DF072B
:101C90001AC0193419F484E693E013C0112399F0A3
:101CA00084E693E00E94D207812F0E94450B809129
:101CB000180A882341F01092180A0E947B0288EDCE
:101CC00093E00E94D20780916009813079F41092EC
:101CD00060092F9AC6010E94D50086EE93E00E940B
:101CE000D207C60160E10E94710520C080916009A1
:101CF0008230E9F4109260092F9AC6010E94D50043
:101D000089EE93E00E94D20786018EEE93E00E9456
:101D1000D207F80181918F0190E00E9408080A150E
:101D20001B0599F787EC93E00E94D2072F988091CA
:101D30006109882309F46ACF8091170A882309F47E
:101D400065CF8091DF07813009F041C080EF93E0DB
:101D50000E94D2078BEF9CE00E94D20787EC93E0B1
:101D60000E94D20789EF93E00E94D2078AE090E0B8
:101D70000E9408088EE993E00E94D2078BED9CE058
:101D80000E94D20787EC93E00E94D20700E010E0A7
:101D9000EE24FF2483EC93E00E94D207C8010E9446
:101DA00008088EE993E00E94D207C7018556944F38
:101DB0000E94D20787EC93E00E94D2070F5F1F4F6B
:101DC00080E290E0E80EF91E0A30110519F7109232
:101DD00061098EEF93E00E94D20700E010E08EEEE2
:101DE00093E00E94D207F801EE0FFF1FE957F44F6E
:101DF000808191810E9408080F5F1F4F00311105FB
:101E000071F782E094E00E94D20700E010E08EEECD
:101E100093E00E94D207F801EE0FFF1FE55EF24F3C
:101E2000808191810E9408080F5F1F4F00321105C9
:101E300071F787EC93E00E94D20788E094E00E945B
:101E4000D2078091710890E00E9408088EEE93E01E
:101E50000E94D2078091720890E00E94080887ECE7
:101E600093E00E94D2078CE094E00E94D207809118
:101E70006509909166090E9408088EEE93E00E9421
:101E8000D2078091F80990E00E9408088EEE93E056
:101E90000E94D2078091F90990E00E9408088EEE16
:101EA00093E00E94D2078091F70990E00E94080811
:101EB0008EEE93E00E94D2078091640990E00E9428
:101EC00008088EEE93E00E94D20780917F0B9091DC
:101ED000800BA091810BB091820B0E9408088EEEBE
:101EE00093E00E94D2078091970B9091980B0E94EB
:101EF000080887EC93E00E94D20788CE97FB092E52
:101F000007260AD077FD04D049D006D000201AF465
:101F1000709561957F4F0895F6F7909581959F4F45
:101F20000895A1E21A2EAA1BBB1BFD010DC0AA1F1A
:101F3000BB1FEE1FFF1FA217B307E407F50720F032
:101F4000A21BB30BE40BF50B661F771F881F991FAD
:101F50001A9469F760957095809590959B01AC01F6
:101F6000BD01CF01089597FB092E05260ED057FD20
:101F700004D0D7DF0AD0001C38F450954095309536
:101F800021953F4F4F4F5F4F0895F6F790958095FD
:101F9000709561957F4F8F4F9F4F0895AA1BBB1B74
:101FA00051E107C0AA1FBB1FA617B70710F0A61B59
:101FB000B70B881F991F5A95A9F780959095BC017A
:101FC000CD010895FB01DC0102C001900D9241504A
:101FD0005040D8F70895FB01DC010D900020E9F78F
:101FE000119701900D920020E1F70895FB01DC01AB
:101FF00001900D920020E1F70895DC01CB01FC0176
:10200000F999FECF06C0F2BDE1BDF89A319600B451
:102010000D9241505040B8F70895DC01CB0103C048
:102020002D910E94181041505040D0F70895262F4E
:10203000F999FECF1FBA92BD81BD20BD0FB6F894AD
:0E204000FA9AF99A0FBE01960895F894FFCF10
:10204E00526561645F53657475703A20000A0D0025
:10205E0057726F6E672045454D414749433A200000
:10206E002F00AA0000000000000000000000000089
:10207E000000000000000000000000000000000052
:10208E0000000000640064006400640064006400EA
:10209E006400640009120D0810040B0E02140701EF
:1020AE000F050C0009120D0810040B0E0214070187
:1020BE000F050C000A0A0A0A0A0A0A0A0A0A0A0A7A
:1020CE000A0A0A0A141414141414141414141414EA
:1020DE00141414141E1E1E1E1E1E1E1E1E1E1E1E3A
:1020EE001E1E1E1E646464646464646464646464BA
:1020FE0064646464000102030405060708090A0B00
:10210E000C0D0E0F0E0F14150C100B191A111612B2
:10211E000D171318110C1A150F10130B0E180D1690
:10212E001719121414120D0F181316110C1A100B76
:10213E000E15191716130E140F181510190B0C1A5D
:10214E00120D171115101317120E0C1A0B0F110D6D
:10215E00161814190E0F14150C100B191A1116123D
:10216E000D17131819110C1A150B140F1810120E37
:10217E00170D13161613180D170F100B190E121527
:10218E0014110C1A0E17120F110C1A1510160B141F
:10219E0019130D180B0C0D0E0F101112131415161A
:1021AE001718191A0A0D535953494E464F3A7A6960
:1021BE00676269742F74782D70706D2F6D657368FA
:1021CE006E65746963732F302E382D313331303094
:1021DE0036303939360A0D004D543A002F003A0088
:1021EE0020200A0D002D2D2D2D2D2D2D2D2D2D2D9B
:1021FE002D2D2D2D2D2D2D2D2D2D0A0D0020003E9A
:10220E00003D004D453A000A0D0072636F70656E19
:10221E0032342D74780A0D0053657475702D536128
:10222E007665640A0D005353005343414E003B0044
:10223E00535953494E464F3A00524D543A00434873
:10224E0056000A0D54454C0041433B004554433B58
:10225E00000000C1C081C1400101C3C00380024122
:10226E00C201C6C006800741C70005C1C581C44072
:10227E000401CCC00C800D41CD000FC1CF81CE40EA
:10228E000E000AC1CA81CB400B01C9C009800841AA
:10229E00C801D8C018801941D9001BC1DB81DA40B2
:1022AE001A001EC1DE81DF401F01DDC01D801C41F2
:1022BE00DC0014C1D481D5401501D7C0178016415A
:1022CE00D601D2C012801341D30011C1D181D040AA
:1022DE001001F0C030803141F10033C1F381F24082
:1022EE00320036C1F681F7403701F5C035803441F2
:1022FE00F4003CC1FC81FD403D01FFC03F803E41EA
:10230E00FE01FAC03A803B41FB0039C1F981F84029
:10231E00380028C1E881E9402901EBC02B802A4111
:10232E00EA01EEC02E802F41EF002DC1ED81EC4071
:10233E002C01E4C024802541E50027C1E781E64059
:10234E00260022C1E281E3402301E1C02180204129
:10235E00E001A0C060806141A10063C1A381A240E1
:10236E00620066C1A681A7406701A5C06580644171
:10237E00A4006CC1AC81AD406D01AFC06F806E41E9
:10238E00AE01AAC06A806B41AB0069C1A981A840A9
:10239E00680078C1B881B9407901BBC07B807A41B1
:1023AE00BA01BEC07E807F41BF007DC1BD81BC40F1
:1023BE007C01B4C074807541B50077C1B781B64059
:1023CE00760072C1B281B3407301B1C071807041A9
:1023DE00B00050C190819140510193C05380524141
:1023EE00920196C056805741970055C195819440F1
:1023FE0054019CC05C805D419D005FC19F819E40E9
:10240E005E005AC19A819B405B0199C05980584128
:10241E00980188C04880494189004BC18B818A4010
:10242E004A004EC18E818F404F018DC04D804C4170
:10243E008C0044C184818540450187C04780464158
:10244E00860182C042804341830041C18181804028
:10245E004001030303030303030303030303020304
:10246E000303030203030303FD09010A020A030A1D
:10247E00040A050A060A070A080A090A0A0A0B0AC2
:10248E000C0A0D0A0F0A100A110A120A130A150A6B
:10249E00160A170A180A6964007461626C65007482
:1024AE00696D657461626C65006C697374656E5FED
:1024BE006265666F72655F74616C6B006C62745FEF
:1024CE006C696D697400727373695F7761726E699E
:1024DE006E67006C71695F7761726E696E6700700E
:1024EE00706D5F696E0070706D5F73796E630073EF
:1024FE00657269616C5F73796E63006D756C74697A
:10250E005F6368616E6E656C006D756C74695F6398
:10251E0068616E6E656C73006D756C74695F6D735A
:10252E00796E635F6E756D006D756C74695F6D733A
:10253E00796E635F6C656E006D756C74695F636850
:10254E00616E6E656C6D6170006D756C7469325F75
:10255E006368616E6E656C006D756C7469325F6375
:10256E0068616E6E656C73006D756C7469325F6D4B
:10257E0073796E635F6E756D006D756C7469325F25
:10258E006D73796E635F6C656E006D756C74693218
:10259E005F6368616E6E656C6D6170006D656E7502
:1025AE005F6C656E006373765F6F75747075740023
:1025BE007361766500560659065F0669067C0686C7
:1025CE000693069F06A606AF06BB06C906D806E802
:1025DE0006F80609071807280739074A075C076532
:1025EE00077007476C6F62616C00496E70757400FE
:1025FE004D756C746970726F70004D756C74697086
:10260E00726F7032004D656E7500A307AA07B00792
:10261E00BA07C50700070A0F1407030505030201D1
:10262E00010101010101010101010101010101018C
:10263E00010101010101010101010101010101017C
:10264E00010101010101010101010101010101016C
:10265E00010101010101010101010101010101015C
:10266E00010101010101010101010101010101014C
:10267E00010101010101010101010101010101013C
:10268E00010101010101010101010101010101012C
:10269E00010101010101010101010101010101011C
:0C26AE0001010101010101010101FF0017
:00000001FF
